:020000040000FA
:100000008B1307309F0083120030850007309F005C
:10001000BF3086008316403086001F308500831273
:10002000861206126520A30A861206126B20061F8E
:1000300017288616061271207120712071207120F8
:10004000061BA415061FA411861206126B20861229
:10005000061671207120712071207120061B241555
:10006000061F24118612061224193D28A41D4928B2
:1000700006108614061586111328A41944280614A0
:10008000861006118615132806148610061586118B
:10009000132806108610061186116B200610861490
:1000A000061186156520231C592806108610061196
:1000B000861523185F280610861406118611652000
:1000C000061486100615861113280530A2006B2031
:1000D000A20B67280800A001A0037120A00B6D28C7
:0C00E0000800A101A103A10B7328080077
:02400E00613F10
:00000001FF
